:1000000000308A002C2800002230840000080319E8
:1000100018280130F800F701F70B0C28F80B0B2813
:100020004A30F700F70B122800000000800B092867
:1000300000341230A302031C2B2823308400FC3030
:1000400080050310800C800C000803192B28292838
:100050000000800B2828003484011F30830583169C
:100060001F129F121B0880399B0007309C001C0840
:1000700083120D13603083168F001F129F121B080E
:1000800080399B0083121F10941283160611861468
:100090000612003083129400831694000108C739B9
:1000A00008388100831290010030F800920000307F
:1000B0008316920007309C0005080330F700F70B09
:1000C0005F281C0883120D1383169D0106158312E9
:1000D000061DB82883168610831286140130A200EC
:1000E00004200230A200F730A3001920A20B7328CD
:1000F0008316861083128610831685118312851548
:100100000130A20004200230A200F730A300192021
:10011000A20B85288316851183128511831605117C
:10012000831205150130A20004200230A200F7302E
:10013000A3001920A20B972883160511831205111D
:1001400083160510831205140130A200042002302A
:10015000A200F730A3001920A20BA92883160510CE
:10016000831205100A30A200042083166628831229
:1001700083160615831206192A29A1012108633C5A
:10018000031CF32883168610831286140130A20004
:10019000042083168610831286108316851183121D
:1001A00085150130A2000420831685118312851164
:1001B00083160511831205150130A2000420831651
:1001C00005118312051183160510831205140130E1
:1001D000A200042083160510831205100A30A20025
:1001E0000420A10ABE28A1012108633C031C29297F
:1001F00083168610831286140230A2000420831610
:10020000861083128610831685118312851502309D
:10021000A20004208316851183128511831605110F
:10022000831205150230A2000420831605118312E3
:10023000051183160510831205140230A200042054
:1002400083160510831205100A30A2000420A10AAB
:0A025000F428B8288316662863001E
:04400E00F83FFF3F39
:00000001FF
